:060000008A150A16002813
:10000800FF00030E83018316EB000A08ED008A0146
:1000180070088312A4007108A3007208A2000408E3
:10002800A50083168C1E7A2883128C1E7A28981CA9
:100038002E2818121A08F200181603171008013E85
:10004800F00000300318013E1107F100700890001D
:10005800710891000313181D432898139817031764
:100068001008013EF00000300318013E1107F100AE
:10007800700890007108910003131A08F2001A081A
:10008800F20072080D3A0319552880304C06F0002A
:1000980080307002031D522840304B020318552847
:1000A80064288316E01683124B08A03E8400800162
:1000B8004B08C9004C08CA00CB01CC01F2017928D1
:1000C8004B08A03E8400720880004B08C9004C0809
:1000D800CA004B08013EF00000300318013E4C07EF
:1000E800F1007008CB007108CC008C128B1E9E2882
:1000F8000B1D9E2883120B113C3081006208013EC3
:10010800F00000300318013E6307F1007008E200B8
:100118007108E30080306306F00080307002031D30
:10012800972864306202031C9E2883166015831288
:10013800E201E30183122408F0002308F1002208F9
:10014800F2002508840083166D088A006B0E830070
:06015800FF0E7F0E0900FE
:08015E00FA1FF2130030080043
:10016600FB14FB1FBD28FF30F300F200F100F00086
:08017600FA0DF20CFF30080045
:10017E007B15FB1FC9280130F300F201F101F001DC
:08018E00FA0DF20CFF3008002D
:0E019600F201F101F001F801F3010030080060
:1001A400243083120313FC00B530FD00FD0BD82866
:0A01B400FC0BD82800000000080032
:1001BE007C181529FC18E6287C193429DF28A101A2
:1001CE007208031D06297108F2007008F100780804
:1001DE00F000F801A1157208031D06297108F2003E
:1001EE007008F100F001A11121167208031D0629F5
:1001FE007108F200F101A1157208031928292108CE
:10020E00F302031D031C2C290310F21B1529F80DF4
:10021E00F00DF10DF20DF30B0C292C297B1B701C2C
:10022E003029F81F3029F00A0319F10A0319F20ACE
:10023E00031D3029F20CF10CF00CF30A03193429CA
:10024E0030290130FC00CB2037290230FC00BF20C2
:10025E0037290430FC00AF2037290830FC00B320CA
:04026E000000080084
:0E027200533083120313FD00FD0B3D290800DD
:0C0280000000000000000000000008006A
:10028C00A1017208031D5B297108F2007008F100CE
:10029C00F001A1157208031D5B297108F200F10130
:1002AC00A11121167208031969292108F302031DF3
:1002BC00031C6D290310F21B7129F00DF10DF20DC9
:1002CC00F30B61296D290130FC00CB20742902301D
:0E02DC00FC00BF2074290430FC00AF20080095
:1002EA0083120317B41B7B2986117C298615341BBC
:1002FA008029061181290615B41A852986108629AE
:10030A008614341A8A2906108B29061483160313B5
:10031A006C189229831285159429831285118514E4
:10032A00402185100317B4199C2986119D29861529
:10033A003419A1290611A2290615B418A62986106E
:10034A00A72986143418AB290610AC29061483167B
:10035A0003136C18B32983128515B52983128511E5
:10036A0085144021851083166C1CBD29D220BE2914
:04037A00392108001D
:10037E008312031372087606A100F801F9017308BF
:10038E007702031CE2297708FD007308F7007D0849
:10039E00F3007608FD007208F6007D08F20075087D
:1003AE00FD007108F5007D08F1007408FD0070086D
:1003BE00F4007D08F000770803195B2A7208FA0032
:1003CE00F217F61777087302F7000319152A08308B
:1003DE007702031C0B2AF7007408F9007508F40065
:1003EE007608F500F60108307702031C0B2AF70099
:1003FE007408F9007508F400F50108307702031C43
:10040E000B2A7A08F2005B2A77080319152A0310C3
:10041E00F60CF50CF40CF90CF70B0E2AA11F222A80
:10042E00F909F409F509F609F90A0319F40A031989
:10043E00F50A0319F60A7908F80774080318740FF9
:10044E00F00775080318750FF10776080318760F75
:10045E00F207A11B3B2A031C4B2AF20CF10CF00CE9
:10046E00F80CF30F4B2A572A03184F2AF809F009F4
:10047E00F109F209F80A0319F00A0319F10A03192E
:10048E00F20A8030FA06532A0130FC00DF205D2A82
:10049E000230FC00DF205D2A0430FC0046215D2A7C
:1004AE000830FC00B3205D2A0030FC00000008007C
:1004BE008316031314196D2A1F301105F1007108EC
:1004CE00003A031D6D2A0130F0006E2AF00108007B
:0604DE00FB15FF300800D1
:1004E4007B14FB1F7D2AF201FA1FFF30F200F1009A
:0A04F400F000FA0DF20CFF300800D2
:1004FE00831603139818852A00007F2A8312031788
:08050E003208031399000800F4
:1005160083120313F8010830FC00700DF80D7408FF
:10052600F8020318982AF8070310F00DFC0B902A1E
:020536000800BB
:1005380083120313F801F9011030FC00710DF80D56
:10054800F90D7408F8027508031C750FF9020318F1
:10055800B42A7408F80775080318750FF90703100B
:0A056800F00DF10DFC0BA22A0800B3
:1005720083120313FB017308031D77080319102B61
:1005820072087606FA007708F3077E30031CCD2A3C
:10059200F3020318132BD02AF302031C162B720842
:1005A200F8007108FC007008FD00F817F617031038
:1005B200F201F101F0011830A1007D1CEA2A740851
:1005C200F00775080318750FF10776080318760F00
:1005D200F207F20CF10CF00CF80CFC0CFD0C031001
:1005E200A10BDE2AF21BFA2AF80DF00DF10DF20D25
:1005F200F3037B1B701C0C2BF81F0C2BF00A031946
:10060200F10A0319F20A031D0C2BF20CF10CF00C87
:10061200F30A0319132BFA1FF2130030182B0130BF
:10062200CB20182B0230B320182B0430BF2000003F
:020632000800BE
:10063400710DF80DF90D7408F8027508031C750F97
:10064400F902F00DF10D0F30FC00710DF80DF90DEC
:100654007408701C332BF8027508031C750FF9021B
:10066400382BF80775080318750FF907F00DF10D0D
:10067400FC0B272B7018442B7408F8077508031813
:08068400750FF90700000800E2
:10068C00831203173208393C031C532B30303202CF
:0E069C00031C532B0130F000542BF00108001A
:0C06AA00831203138030F606BF21080005
:1006B60083120313FB01FA01F9018030F800F10CF3
:1006C600F00C031C6F2B7408F90775080318750FD7
:1006D600FA070318FB0A0310F01F772B7408FA07B2
:1006E60075080318750FFB07FB0CFA0CF90CF80CD0
:1006F600031C622B7B08F3007A08F2007908F100EC
:060706007808F000080075
:0E070C00831603139114911C8C2B892B08006B
:10071A00831203138C118316911583128C19962B4D
:10072A00922B1308F10003173208003A031DA12B7C
:10073A00831603139116A42B8316031391128312A3
:10074A008C118316111683128C19AC2BA82B7108E5
:04075A00F0000800A3
:08075E008316031311150800B6
:0E076600831603136F088A006E0882000800D5
:10077400831203137408003A031DD52B7508003A3D
:10078400031DD52B7608003A031DD52B7708003AB4
:10079400031DD52BFF30F000FF30F1007F30F20055
:1007A400FF30F300702C8312031377080319642CB1
:1007B40073080319672C720876068039FA00F21759
:1007C400F617A1017208F8007108FC007008FD001A
:1007D4007408FD027508031C750FFC027608031CDF
:1007E400760FF802F801FC01FD01031C002C031034
:1007F400F20CF10CF00CF80C0130A1007708F302B4
:10080400031C0A2C7E302107F30703186A2C0F2CD3
:100814007E302107F307031C6D2C1830FA07FD0DF9
:10082400FC0DF80DF00DF10DF20DA10D7408F002A0
:100834007508031C750FF1027608031C760FF2028B
:10084400760DA104211C282C7D14332C7408F00788
:1008540075080318750FF10776080318760AF2076E
:100864007D10FA031F307A05031D112C7B1B7D1CA0
:100874005A2C0310F00DF10DF20DA10D7408F002C5
:100884007508031C750FF1027608031C760FF2023B
:10089400760D21040139FD070318FC0A0319F80A2F
:1008A400031D5A2CF80CFC0CFD0CF30A03196A2CDA
:1008B400FA1FF8137808F2007C08F1007D08F000B4
:1008C40000306F2C01306F226F2C0230CB206F2C44
:0E08D4000430B3206F2C0830BF200000080055
:1008E200831203137008F8007108F000F101F2019D
:1008F200F301FB01FC019630F300FA01F01F872C93
:10090200F809F009F80A0319F00AFA177008F10059
:0C0912007808F000F801F201462108000E
:10091E0083120313FB0173080319CC2C7208FA001F
:10092E00F2178E30F302F31FCF2CF309F30A0830BF
:10093E007302031CB22CF300F10D7208F100F201E8
:10094E0008307302031CB22CF300F10DF101730891
:10095E00031D0310BA2C73080319BA2C0310F20CE2
:10096E00F10CF30BB52C7B1B711CC42C031CC42C7B
:10097E00F10A0319F20AF21BDB2CFA1FDE2CF20924
:10098E00F109F10A0319F20ADE2CF201F101DE2C53
:10099E007B14FB1FE12CF201FA1FE12CFF30F20059
:1009AE00F100FA0DF20CE12C0130FC00E32C0030CA
:1009BE00FC00E32CFF30FC00FC080319E72C72222C
:0A09CE007108F0007208F100080043
:1009D800831603136C10831203173208B4007521B1
:0609E80083166C140800E8
:1009EE0083120313FA017308031D7A147708031D8B
:1009FE00FA147A080319432D033A03190E2D7A18A7
:100A0E000B2DF61F412D3F2DF21F3F2D412D72084C
:100A1E008039FA00F21376088039F6137A06031934
:100A2E001C2D7A0803193F2D412D770873020319E7
:100A3E00232D031C372D3B2D7608720203192A2D08
:100A4E00031C372D3B2D750871020319312D031C24
:100A5E00372D3B2D740870020319432D03183B2DBF
:100A6E00FA080319412D3F2DFA0803193F2D412D88
:100A7E0003140800031008000314031508000800EF
:100A8E0083120317B201B3013308123C031D512D1B
:100A9E0032088E3C031C5E2D5F2270080319582D00
:100AAE005E2D83120317B20A0319B30A4B2D83125C
:100ABE00031712303302031D662D8F303202031CD2
:100ACE006B2D7B30F000722D831603131114111C45
:080ADE00712D6E2DF0010800DE
:100AE600831203138C110317320803139300831622
:100AF600141D7E2D7A2D83128C19822D7E2D831640
:100B0600111B872DF0018A2D11150230F000080007
:100B160083120313FB01FA01F901F801A001730D19
:100B2600F80D7408F8027508031C750FF9027608AB
:100B3600031C760FFA027708031C770FFB020001ED
:100B4600031C0130A002F30D0730FC00730DF80DF5
:100B5600F90DFA0DFB0DA00D7408731CC42DF802D7
:100B66007508031C750FF9027608031C760FFA0246
:100B76007708031C770FFB020001031C0130A0025B
:100B8600D52DF80775080318750FF90776080318A9
:100B9600760FFA0777080318770FFB07000103188B
:100BA6000130A007F30DFC0BA92D720DF80DF90D00
:100BB600FA0DFB0DA00D7408731CF32DF8027508D1
:100BC600031C750FF9027608031C760FFA027708E4
:100BD600031C770FFB020001031C0130A002042E48
:100BE600F80775080318750FF90776080318760FC6
:100BF600FA0777080318770FFB070001031801307F
:100C0600A007F20D0730FC00720DF80DF90DFA0D74
:100C1600FB0DA00D7408721C222EF8027508031C29
:100C2600750FF9027608031C760FFA027708031C83
:100C3600770FFB020001031C0130A002332EF807D8
:100C460075080318750FF90776080318760FFA0763
:100C560077080318770FFB07000103180130A00778
:100C6600F20DFC0B072E710DF80DF90DFA0DFB0DAB
:100C7600A00D7408721C512EF8027508031C750F1E
:100C8600F9027608031C760FFA027708031C770F21
:100C9600FB020001031C0130A002622EF807750852
:100CA6000318750FF90776080318760FFA07770801
:100CB6000318770FFB07000103180130A007F10D99
:100CC6000730FC00710DF80DF90DFA0DFB0DA00DA6
:100CD6007408711C802EF8027508031C750FF90242
:100CE6007608031C760FFA027708031C770FFB02BF
:100CF6000001031C0130A002912EF80775080318A5
:100D0600750FF90776080318760FFA0777080318A0
:100D1600770FFB07000103180130A007F10DFC0B4C
:100D2600652E700DF80DF90DFA0DFB0DA00D74086A
:100D3600711CAF2EF8027508031C750FF9027608B0
:100D4600031C760FFA027708031C770FFB020001DB
:100D5600031C0130A002C02EF80775080318750F92
:100D6600F90776080318760FFA0777080318770F3E
:100D7600FB07000103180130A007F00D0730FC0047
:100D8600700DF80DF90DFA0DFB0DA00D7408701C11
:100D9600DE2EF8027508031C750FF9027608031C8F
:100DA600760FFA027708031C770FFB020001031C7B
:100DB6000130A002EF2EF80775080318750FF90722
:100DC60076080318760FFA0777080318770FFB07DC
:100DD600000103180130A007F00DFC0BC32E70189C
:100DE600022F7408F80775080318750FF9077608B7
:100DF6000318760FFA0777080318770FFB07080022
:100E060083120317A1011F0884000008A000200810
:100E1600003A0319192F2008B2007F220317A10AEE
:0E0E260021081F0784000008A0000A2F080002
:100E3400831203171F08F2007208F000F20A700808
:100E4400840000080319272F1E2F1F087202F000C8
:0C0E54000130F002F101031CF103080062
:100E6000831203171F0884000008A000A1010030AE
:100E7000A10000302106031D3F2F2030200603195A
:100E80004A2F00302106031D472F09302006031981
:100E90004A2F4C2F9F0A302FA201A301A401A501C4
:100EA00000302106031D562F2D302006031D5D2F17
:100EB000A40A0319A50A9F0A662F00302106031D04
:100EC000632F2B302006031D662F9F0A1F08840006
:100ED0000008A000A1010030A1002008B2004623B4
:100EE000700803198F2F2208F0002308F1000A3040
:100EF000F4000030F5005B23303003172002F200CD
:100F00000030031C013E2102F30072087007A200AA
:100F100071080318013E7307A3009F0A662F240877
:100F2000250403199C2F2208003CF0002308031C11
:100F3000013EF101F102A02F2208F0002308F10088
:020F40000800A7
:100F4200831203171F085A3C031CAE2F41301F02A5
:0E0F5200031CAE2F0130F000AF2FF00108009D
:100F6000FF30831203171F058D0083168C130C149A
:100F70000C140C1CBC2FB82F83120C08F0000800B6
:100F800083120317A0011F08093C0318E42F0A303D
:100F9000F4001F08F0008B2270080317A0007008EF
:100FA000A000A00D2010A00D2010A00D2010A00D5D
:100FB00020100A30F4001F08F0008B227808F0009F
:100FC00070080317A004E62F1F08A0002008F000F7
:020FD000080017
:100FD2000A3083120317B2007F220D300317B200CA
:040FE2007F22080062
:0C0FE600831203139501171297120800E4
:1010000012288030831203179F002528C0309F00CC
:10101000252894309F002528D4309F002528803033
:101020009F002528831203171F08013A031901287E
:101030001F08023A031906281F08033A0319092852
:101040001F08043A03190C280F282003F0001F087A
:10105000F00770089F007008B4008A1175218A1586
:1010600083166C1083120317A20122082107840043
:101070000008031947282208210784000008B2004D
:101080008A11EC248A1583120317A20A35288316C5
:0610900003136C140800BC
:10109600831203171F0883160313EE008312031728
:1010A600200883160313EF008A11B3238A150A1248
:1010B600F000700803197A28831203171F08831695
:1010C6000313EE0083120317200883160313EF00A1
:1010D6008A11B3238A150A1283120317B2008A11E2
:1010E6007F228A1503179F0A0319A00A4B280800B6
:1010F600831203172308A5002408003C031C882834
:101106000730F4000030F5009F282408163C031829
:1011160091281730F2000030F3009B282408013E86
:10112600F000F1010318F10A7008F2007108F300EB
:101136007208F4007308F5007408AC007508AD0079
:10114600A601A701F401F501F601F7011F08F00059
:101156002008F1002108F2002208F3008A11F72482
:101166008A15013003180030F00070080319C928E9
:101176000317230884002D308000A30A00309F0641
:101186000030A0068030A1060030A20603171F0813
:10119600F4002008F5002108F6002208F700F00107
:1011A600F101F201F3018A11F7248A1501300318BF
:1011B6000030F000700803191D290030F4000030DB
:1011C600F5000030F6007F30F70003171F08F00027
:1011D6002008F1002108F2002208F3008A11F72402
:1011E6008A15013003180030F000700803191D2914
:1011F60003171F08F0002008F1002108F20022085A
:10120600F3000030F4000030F5002030F6008230A4
:10121600F7008A11B9228A15700803179F00710812
:10122600A0007208A1007308A2000130A602031CE8
:10123600A703E02803170030F4000030F500203043
:10124600F6008230F7001F08F0002008F1002108A0
:10125600F2002208F3008A11F7248A150130031CD4
:101266000030F0007008031959290030F4000030EE
:10127600F5002030F6008230F70003171F08F00053
:101286002008F1002108F2002208F3008A11BA238F
:101296008A15700803179F007108A0007208A10044
:1012A6007308A200A60A0319A70A1D290317260810
:1012B600AC0727080318013EAD070130A80000302F
:1012C600A9000130F0000030F1008A1171248A155E
:1012D60070080317AE007108AF007208B0007308FB
:1012E600B10080302906F00080302D067002031D03
:1012F6007E292C0828020318A0290030F4000030AB
:10130600F5002030F6008230F7002E08F0002F0896
:10131600F1003008F2003108F3008A11BA238A1569
:1013260070080317AE007108AF007208B0007308AA
:10133600B100A80A0319A90A74290030F400003084
:10134600F5000030F6008030F7002E08F0002F0878
:10135600F1003008F2003108F3008A11BA238A1529
:1013660003171F08F4002008F5002108F6002208DC
:10137600F7008A11BF218A15700803179F007108AC
:10138600A0007208A1007308A2000030F40000302B
:10139600F5002030F6008230F7008A11F7248A150E
:1013A6000130031C0030F00070080319E6290030F4
:1013B60003179F000030A0000030A1007F30A2007C
:1013C600A60A0319A70A031780302706F000803003
:1013D6007002031DF029003026020318272A23086D
:1013E600840030308000A30A230884002E30800059
:1013F600A30A80302D06F00080307002031D052AF6
:1014060000302C0203180D2A2C08A602031CA70381
:101416002D08A702FF30A800FF30A900803027065C
:10142600F000803029067002031D1B2A28082602B8
:101436000318272A2308840030308000A30A0130CD
:10144600A802031CA903112AA801A90180302906B4
:10145600F00080302D067002031D332A2C08280266
:1014660003189D2A1F08F0002008F1002108F20049
:101476002208F3008A118F248A1570080317AA0020
:101486007108AB003030F007230884007008800034
:10149600A30A29082706031D522A26082806031D23
:1014A600592A230884002E308000A30A2A08F00057
:1014B6002B08F1008A1171248A1570080317AE00F3
:1014C6007108AF007208B0007308B1007008F4002C
:1014D6007108F5007208F6007308F7001F08F0009F
:1014E6002008F1002108F2002208F3008A11552392
:1014F6008A15700803179F007108A0007208A100E2
:101506007308A2000030F4000030F5002030F60029
:101516008230F7008A11B9228A15700803179F00D6
:101526007108A0007208A1007308A200A80A031996
:10153600A90A292A2308840080012508F00008004A
:1015460083120317A401A50100302502031DAD2A4D
:101556000A3024020318B82A2408230784002030FE
:101566008000A40A0319A50AA72A240823078400D1
:1015760080010130A402031CA50324082307A6004A
:101586000A30F400F501F601F7011F08F000200803
:10159600F1002108F2002208F3008A118B258A1532
:1015A6007808F0007908F1007A08F2007B08F30069
:1015B60030307007F4000317260884007408800092
:1015C6000A30F400F501F601F7011F08F0002008C3
:1015D600F1002108F2002208F3008A118B258A15F2
:1015E600700803179F007108A0007208A100730815
:1015F600A2000030F4007306031D0B2B740872065C
:10160600031D0B2B74087106031D0B2B7008003A83
:10161600031D0E2B132B0130A402031CA503C02AA5
:021626000800BA
:10162800831203137408003A031D232B7508003A2C
:10163800031D232BFF30F0007F30F1007E2B831237
:101648000313FD01F901F80171087004031900344E
:1016580071087506FA00FA1BFD09FB01F51F392B05
:10166800F409F509F40A0319F50AF11F402BF009EA
:10167800F109F00A0319F10A71087504FA00FA1B56
:10168800552B8A111A238A157B186A2BFD1F0034E3
:10169800F009F109F00A0319F10AF809F909F80A39
:1016A8000319F90A0034F51F662BF11B622B710828
:1016B800F9007008F800F101F0014A2BF101F0017E
:1016C800F00A0034F109F009FB0A472BF80A03195C
:1016D800F90A74087802031D4A2B75087902031D5C
:1016E8004A2BF901F801F00A0319F10AF11F4A2BF4
:0616F8000000FF340800B1
:1016FE008A1147258A15A03083120317B2008A116A
:10170E0073258A15831203172008F000F101700863
:10171E00B2008A1173258A15FF30831203171F0535
:10172E00B2008A1173258A15831203172108B2009D
:10173E008A1173258A158A11AF238A152130FC0070
:10174E007630FD00FD0BA92BFC0BA92B0000080029
:10175E008A1147258A15D03083120317B2008A11D9
:10176E0073258A1583120317B2018A1173258A1500
:10177E008A1186238A15D13083120317B2008A117B
:10178E0073258A150730FC007D30FD00FD0BCD2B37
:10179E00FC0BCD2B013083120317B2008A118D235F
:1017AE008A1503171F088400700880000130B200EC
:1017BE008A118D238A150317200884007008800073
:1017CE000130B2008A118D238A1503172108840077
:1017DE00700880000130B2008A118D238A1503171C
:1017EE0022088400700880000130B2008A118D2317
:1017FE008A15031723088400700880000130B20098
:10180E008A118D238A15031724088400700880001E
:10181E00B2018A118D238A150317250884007008DA
:0A182E0080008A11AF238A1508001C
:10183800831203171F087A3C031C292C61301F02EE
:0E184800031C292C0130F0002A2CF0010800AE
:1018560083120317A201053022020318392C22082D
:101866002107840020308000A20A2E2C220821079E
:1018760084008001A20322082107A3000A30F40095
:10188600F5011F08F0002008F1008A119C228A1534
:101896007808F0007908F1003030F00703172308C4
:1018A6008400700880000A30F400F5011F08F0007B
:1018B6002008F1008A119C228A15700803179F00E0
:1018C6007108A00000307106031D6B2C00307006F5
:0C18D600031D6E2C702CA2033E2C080099
:1018E200832C8030831203179F00962CC0309F00F8
:1018F200962C94309F00962CD4309F00962C8030EA
:101902009F00962C831203171F08013A0319722CA9
:101912001F08023A0319772C1F08033A03197A2C7D
:101922001F08043A03197D2C802C2003F0001F08A5
:10193200F00770089F00831603136C14700883125B
:101942000317B4008A1175218A1583166C1083124D
:1019520003172108B4008A1175218A1583166C14A5
:0219620008007B
:10196400831203137008F100F0010830FC007108C1
:10197400F40C0318C12CFC0BBA2CF1010034031035
:10198400C62CF40C0318F107F10CF00CFC0BC32C5F
:02199400080049
:1019960083120317200883160313EE00831203171E
:1019A600210883160313EF008A11B3238A150A123E
:1019B600F00070080319FB2C831203172008831606
:1019C6000313EE0083120317210883160313EF0097
:1019D6008A11B3238A150A12F000831203171F080F
:1019E6008400700880009F0AA00A0319A10ACB2C64
:0C19F600831203171F0884008001080002
:101A020083120317A00120081F078400000803198E
:101A1200162D20081F0784000008B2008A11EC244A
:0C1A22008A1583120317A00A042D080087
:101A2E008A1147258A15D03083120317B2008A1106
:101A3E0073258A1583120317B2018A1173258A152D
:101A4E00803083120317B2008A1173258A15831210
:101A5E004D080317B2008A1173258A1583124E089A
:101A6E000317B2008A1173258A1583125B080317B8
:101A7E00B2008A1173258A1583125C080317B2000F
:101A8E008A1173258A15831259080317B2008A1119
:101A9E0073258A1583125A080317B2008A1173250B
:101AAE008A158A11AF238A158A1147258A15413066
:101ABE0083120313FC00EE30FD00FD0B642DFC0BB6
:101ACE00642D0000D0300317B2008A1173258A15D9
:101ADE0083120317B2018A1173258A158312031715
:101AEE00B2018A1173258A158A11AF238A1508004F
:101AFE00831603131208013EF000F1010318F10AD8
:101B0E00831203171208F400F5018A115B238A155C
:101B1E000630F2007008F4007108F500720803191F
:101B2E009D2DF50CF40CF513FF3E962D0430F100AF
:101B3E007408F00071080319A82DF00D7010FF3E07
:101B4E00A22D30307005F3007408F0007508F10016
:101B5E00F10CF00CF113F10CF00CF1137008950070
:0A1B6E000F30970573089704080074
:101B7800831203137008F8007108F000F101F201F4
:101B8800F301FB01FC019630F300FA017008F10043
:101B98007808F000F801F2018A1146218A15080038
:101BA80002308312031792000030930096019701C8
:101BB800831603138C12A030831203179F008A1117
:101BC8001A278A1570089400710895008316031364
:101BD8002008553A031DA92E013083120317140259
:101BE800F0000030031C013E1502F1007008A03E11
:101BF80084000008F1007108233A031DA92E8030E3
:101C08001506F00080307002031D0C2E15301402EA
:101C18000318A92E3C309F001630A0004B2002303C
:101C28008312031798000030990080301906F000DD
:101C3800803015067002031D232E1408180203189D
:101C48004E2E1808A03E84000008F10071083B3AA7
:101C5800031D4A2E1808A03E8400800116084F3E36
:101C68009A001208A03E9F008A1130278A151A0888
:101C78008400700880001808013E920000300318A4
:101C8800013E19079300960A0319970A980A03193F
:101C9800990A192E01301402F0000030031C013E8D
:101CA8001502F1007008A03E8400800116084F3E1E
:101CB8009A001208A03E9F008A1130278A151A0838
:101CC8008400700880000313540803179F008A11CA
:101CD800C0278A1570080313CD00530803179F0007
:101CE8008A11C0278A1570080313CE004F080317FE
:101CF8009F008A11C0278A1570080313DC0050085A
:101D080003179F008A11C0278A1570080313D9008A
:101D1800510803179F008A11C0278A1570080313FA
:101D2800DA00520803179F008A11C0278A15700825
:101D38000313DB001725A0018312031796019701EF
:101D48009001910183160313E012831603138C1676
:021D5800080081
:101D5A00C03083120317B4008A1175218A152E30F8
:101D6A0003179F000630F0000030F1001208F4005B
:101D7A00F5018A115B238A157008A73E0317A00094
:101D8A0015300318013E7107A100CB2402309F00D1
:101D9A000130A0002E30A100002002308312031768
:101DAA009F000630A0002030A10071240230831267
:101DBA0003179F000730A0000A30F4001308F00050
:101DCA008A118B228A15303070070317A1007124FB
:101DDA000230831203179F000830A0000A30F40073
:101DEA001308F0008A118B228A157808F000303027
:101DFA0070070317A10071240230831203179F0092
:101E0A000930A0002F30A100712402308312031779
:101E1A009F000A30A0000A30F4001408F0008A116A
:101E2A008B228A15303070070317A1007124023003
:101E3A00831203179F000B30A0000A30F400140825
:101E4A00F0008A118B228A157808F000303070076A
:101E5A000317A10071240230831203179F000C306C
:101E6A00A0002F30A10071240230831203179F00B3
:101E7A000D30A0003230A100712402308312031702
:101E8A009F000E30A0003030A1007124023083126E
:101E9A0003179F000F30A0000A30F4001508F00065
:101EAA008A118B228A15303070070317A10071241A
:101EBA000230831203179F001030A0000A30F4008A
:101ECA001508F0008A118B228A157808F000303044
:0A1EDA0070070317A100712408002F
:101EE400831603130711831212150C30970408008C
:101EF4008A1147258A15A03083120317B2008A116C
:101F040073258A15831203171308F000F101700872
:101F1400B2008A1173258A15FF3083120317120544
:101F2400B2008A1173258A158A1186238A15A13075
:101F340083120317B2008A1173258A1583120317BB
:101F4400B2018A118D238A157008031794008A112F
:0E1F5400AF238A15831203171408F00008004B
:101F6200831203171208B2008A1146238A157008D9
:101F7200031DCB2F12089F001C247008031DCB2FBA
:101F820012089F008A11A1278A157008031DCB2F02
:0A1F9200F001CD2F0130F00008002F
:101F9C008312031712089F008A11B0278A15700844
:101FAC0093007008003C0318E02F1308B2008A114C
:101FBC007F228A150317920A8230FC00DD30FD0067
:101FCC00FD0BE62FFC0BE62F000000001308003A77
:101FDC000319F52FFF3012020318F52FCE2F08002E
:101FEC0083160313141394130716871538308312B2
:041FFC009400080045
:1020000083120317950196011208073C03180B2849
:10201000F001F1019C28C73003139F050317120834
:10202000F000F00D7010F00D7010F00D70107008D1
:1020300003139F041430FC007930FD00FD0B1E28B3
:10204000FC0B1E2800000000031793019401803050
:102050001406F00080307002031D30282030130277
:1020600003188E2803131F1500001F1D382835285C
:102070001E08F100F00183161E08F0070318F10A8C
:10208000700883120317950771080318013E96071D
:1020900070089F007108A0006930A1008A150A121B
:1020A0002B248A110A1683160313601E80286930B8
:1020B000831203179F000A1203270A160930B20081
:1020C0000A127F220A160830F4000030F5000317C8
:1020D0001308F0001408F1008A150A1214238A115B
:1020E0000A167808F0007908F10000307106031D27
:1020F0007B2800307006031D80280A12E9270A1683
:102100000730FC007D30FD008312FD0B8428FC0BA2
:1021100084280317930A0319940A27280530F2002C
:102120001508F0001608F100720803199C28F10C3C
:0A213000F00CF113FF3E95280800A3
:10213A00803083120317B4000A1275210A162E3052
:10214A0003179F00F930A0000730A1008A150A1270
:10215A00CB248A110A1601309F000130A0002E30CC
:10216A00A1008A150A1200208A110A160130831268
:10217A0003179F000730A0000A30F4001408F0008B
:10218A000A128B220A16303070070317A1008A152B
:10219A000A1271248A110A160130831203179F004A
:1021AA000830A0000A30F4001408F0000A128B224A
:1021BA000A167808F000303070070317A1008A1554
:1021CA000A1271248A110A160130831203179F001A
:1021DA000930A0003A30A1008A150A1271248A1126
:1021EA000A160130831203179F000A30A0000A3032
:1021FA00F4001308F0000A128B220A163030700716
:10220A000317A1008A150A1271248A110A160130CD
:10221A00831203179F000B30A0000A30F400130842
:10222A00F0000A128B220A167808F0003030700784
:10223A000317A1008A150A1271248A110A1601309D
:10224A00831203179F000C30A0003A30A1008A15B0
:10225A000A1271248A110A160130831203179F0089
:10226A000D30A0000A30F4001208F0000A128B2286
:10227A000A16303070070317A1008A150A12712452
:10228A008A110A160130831203179F000E30A0002C
:10229A000A30F4001208F0000A128B220A16780893
:1022AA00F000303070070317A1008A150A12712452
:1022BA008A110A160130831203179F000F30A000FB
:1022CA002030A1008A150A1271248A110A160130D7
:1022DA00831203179F001030A0002030A1008A1536
:0A22EA000A1271248A110A16080076
:1022F40083120313AE01031712089F001308A000F2
:102304001408A1001508A2002E30A3001608A4008A
:102314008A150A127B208A110A162E309F000A128F
:102324001A270A161808F00719080318013EF107BE
:1023340070080E3C9C007108031C013E9D019D0227
:102344009A019B0180301B06F00080301906700250
:10235400031DAE2918081A020318BA291430B40050
:102364000A1275210A1603179A0A03199B0AA4294B
:102374009A019B0180301B06F00080301D0670021C
:10238400031DC6291C081A020318D3292030B200E1
:102394000A12EC240A16831203179A0A03199B0AD9
:1023A400BC292E309F008A150A1201258A110A16AB
:1023B4002030B2000A12EC240A1656308312031796
:0A23C400B2000A12EC240A16080009
:1023CE008312031712088400000899007F30190544
:1023DE00F2007208F000F00CF013F00CF013F00C99
:1023EE00F013F00CF0130A30F4008A150A12B2241E
:1023FE008A110A160F3003171905F1007108F0073C
:10240E0012088400700880001308840000089900E8
:10241E00F0301905F2007208F000F00CF013F00C19
:10242E00F013F00CF013F00CF0130A30F4008A15D0
:10243E000A12B2248A110A160F3003171905F10079
:10244E007108F007130884007008800014088400D7
:10245E000008990030301905F2007208F000F00CF7
:10246E00F013F00CF013F00CF013F00CF0130A3024
:10247E00F4008A150A12B2248A110A160F300317B5
:10248E001905F1007108F007140884007008800027
:10249E001508840007300005F00015088400700848
:1024AE0080001608840000089900F0301905F2002B
:1024BE007208F000F00CF013F00CF013F00CF013A7
:1024CE00F00CF0130A30F4008A150A12B2248A11A5
:1024DE000A160F3003171905F1007108F0071608D8
:1024EE0084007008800017088400000899001030DE
:1024FE001905F2007208F000F00CF013F00CF01356
:10250E00F00CF013F00CF0130A30F4008A150A12D6
:10251E00B2248A110A160F3003171905F10071083B
:10252E00F00717088400700880001808840000085F
:10253E009900F0301905F2007208F000F00CF0135B
:10254E00F00CF013F00CF013F00CF0130A30F40052
:10255E008A150A12B2248A110A160F3003171905AA
:10256E00F1007108F0071808840070088000080058
:10257E0083160313981690308312980083168717CC
:10258E00071383128C1ECE2A1A08F000C82A0800E0
:10259E000A12B3238A110A168000840AEE0A03195E
:0A25AE00EF0AF003031DCF2A080016
:1025B800503083120313D8005930CD001330CE00A9
:1025C8000430DC000630D9000430DB001430DA00B7
:0C25D8008A150A1217258A110A1608003D
:1025E4008130831203139F008E3083169F000800EE
:1025F4008312031799019A0112089B0013089C0087
:1026040014089D0015089E0080301506F0008030E7
:102614007002031D172B00301402031D172B00300A
:102624001302031D172B0030120203183F2B013035
:10263400990000309A00F401F501F601F70112083F
:10264400F0001308F1001408F2001508F3007408F0
:102654009B0075089C0076089D0077089E00700812
:102664009B027108031C710F9C027208031C720FF9
:102674009D027308031C730F9E021B089F001C0815
:10268400A0001D08A1001E08A2001608A3008A15B8
:102694000A12A3228A110A160B3097000030980000
:1026A4001808003C031D582B1708003C0318732B13
:1026B40017081607F20001301702F0000030031C5F
:1026C400013E1802F1007008160784000008F000AB
:1026D400720884007008800001309702031C98037C
:1026E400522B160884002030800019081A0403199C
:1026F400912B970198011708160784000008203AC7
:10270400031D882B970A0319980A7D2B0130970221
:10271400031C98031708160784002D308000080056
:10272400831603138101811281110B110115811488
:0E27340001143C30831281000B118B1208003F
:10274200831203171208F000F00CF013F00CF013D0
:10275200F00CF013F00CF0130030F1003030F00701
:1027620017300318013EF107700883160313EE00B9
:102772007108EF000A12B3238A110A16F0008312BD
:1027820003171308840070088000130AF2000F3048
:102792001205F0000030F1003030F0071730031856
:1027A200013EF107700883160313EE007108EF0073
:1027B2000A12B3238A110A16F00072088400700804
:1027C200800002308312031713078400800108007F
:1027D200203083120313F0004E30F100F201F301B6
:0227E2000800ED
:1027E40083160313851085110610861006118611B1
:1027F40083128510851186110611861006100A129F
:10280400D2200A160A12D2200A160A12D2200A1656
:102814008614061485140A1240210A1685100A1219
:10282400D2200A1685140A1240210A1685100A12AB
:10283400D2200A1685140A1240210A1685100A129B
:10284400D2200A16061085140A1240210A16851091
:102854000A12D2200A1685140A1240210A1685107B
:102864008610861585140A1240210A1685100A124C
:10287400D2200A168611061485140A1240210A165B
:102884008510061085140A1240210A1685100A12B2
:10289400D2200A1685140A1240210A16851006143D
:1028A40085140A1240210A1685100A12D2200A162B
:1028B400061085140A1240210A168510861506157D
:1028C4008614061485140A1240210A1685100A1269
:0A28D400D2200A1683166C140800C7
:1028DE008B135830831203179F004D30A0004E30DB
:1028EE00A1005B30A2005C30A3005930A4005A3026
:1028FE00A5008A150A12AF238A110A1683122C0814
:10290E0003179F0003132D080317A0000313590884
:10291E000317A1008A150A127F238A110A16831241
:10292E00AC0A0319AD0A2C0803179F0003132D08D8
:10293E000317A00003135C080317A1008A150A12DF
:10294E007F238A110A168312AC0A0319AD0A2C08CA
:10295E0003179F0003132D080317A00003134E083F
:10296E000317A1008A150A127F238A110A168312F1
:10297E00AC0A0319AD0A2C0803179F0003132D0888
:10298E000317A00003134D080317A1008A150A129E
:10299E007F238A110A168312AC0A0319AD0A2C087A
:1029AE0003179F0003132D080317A00003135808E5
:1029BE000317A1008A150A127F238A110A168312A1
:1029CE00AC0A0319AD0A2C0803179F0003132D0838
:1029DE000317A0000D30A1008A150A127F238A1159
:0E29EE000A168312AC0A0319AD0A8B170800F3
:10300000743083120313A6001530A7004030A800C7
:103010001530A900FE30AA001430AB000E30831624
:103020009F00F130850083128511051185108516EA
:10303000051607138717FA308316870088010130B9
:1030400083128800F0308316860083128601803058
:103050008316810083128813E401E50100306502C4
:10306000031D342850306402031845288317640870
:10307000A03E84006408F000F00D7010700880001D
:103080008313E40A0319E50A2E2881308316990078
:1030900018158A11BF228A1507100C300317B200C9
:1030A0008A110A127F228A150A161A30FB005E3036
:1030B000FC006E30FD00FD0B5B28FC0B5B28FB0B5E
:1030C0005B2800000C300317B2008A110A127F221D
:1030D0008A150A161A30FB005E30FC006E30FD00C7
:1030E000FD0B7028FC0B7028FB0B702800002608D5
:1030F00003179F00031327080317A0000A124B2091
:103100000A1683120313280803179F0003132908C4
:103110000317A0000A124B200A16831203132A0871
:1031200003179F0003132B080317A0000A124B205C
:103130000A1660308312031792000A12CE270A166D
:103140008A11E9238A157008DD007108DE00720813
:10315000DF007308E000403003179F001730A00025
:103160000A124B200A16831203135D0803179200FC
:1031700003135E080317930003135F0803179400FB
:1031800003136008031795002E3096008A11FA2267
:103190008A152E309F008A110A1203278A150A16F3
:1031A0008A110A12E9278A150A164B3003179F0065
:1031B0001730A0000A124B200A1683120313881638
:1031C0008A11F2238A15803083120317B4008A1102
:1031D0000A1275218A150A162E3003179F00FD303A
:1031E000A0001630A1000A12CB240A162E309F0030
:1031F0000A1201250A163330FB00BB30FC00DF3019
:10320000FD00FD0B0129FC0B0129FB0B012900002E
:1032100000000F309F001630A0000A124B200A1643
:10322000803083120317B4008A110A1275218A159F
:103230000A162E3003179F00EC30A0001630A100B4
:103240000A12CB240A162E309F000A1201250A16F4
:103250001A30FB005E30FC006E30FD00FD0B2E29A5
:10326000FC0B2E29FB0B2E29000056309F00173037
:10327000A0000A124B200A168A11F2228A15831224
:10328000AC01AD010C300317B4008A110A1275218C
:103290008A150A16523003179F001630A0000A1232
:1032A0004B200A160C308316031393000A12F627DC
:1032B0000A162E3003179F00DB30A0001630A10045
:1032C0000A12CB240A162E309F000A1201250A1674
:1032D0003330FB00BB30FC00DF30FD00FD0B6E29FE
:1032E000FC0B6E29FB0B6E29000000000313851AEE
:1032F0007B2908137C29081701300317B4008A11B1
:103300000A1275218A150A160330FB008A30FC0068
:103310005530FD00FD0B8A29FC0B8A29FB0B8A29FD
:103320000000000080300317B4008A110A127521D2
:103330008A150A16851AC6292E3003179F001F30DA
:10334000A0001730A1000A12CB240A162E309F00CD
:103350000A1201250A16D7309F001530A0000A1264
:103360004B200A16333083120313FB00BB30FC00E2
:10337000DF30FD00FD0BBA29FC0BBA29FB0BBA2983
:10338000000000008A11DC228A15DD292E3083120C
:1033900003179F000E30A0001730A1000A12CB24A3
:1033A0000A162E309F000A1201250A16F4309F00DB
:1033B0001530A0000A124B200A1633308312031373
:1033C000FB00BB30FC00DF30FD00FD0BE529FC0BF2
:1033D000E529FB0BE5290000000080300317B4004D
:1033E0008A110A1275218A150A16583003179F0090
:1033F0004D30A0004E30A1005B30A2005C30A30035
:103400005930A4005A30A5000A12AF230A165830CA
:103410008312031792004D3093004E3094005B30BE
:1034200095005C309600593097005A3098008A1108
:10343000E7218A15031358080317920003134D0858
:103440000317930003134E08031794008A119D205D
:103450008A1583125B080317920003135C08031795
:103460009300031359080317940003135A08031712
:1034700095000A12AD260A166130831203179F00C9
:103480001730A0000A124B200A1683120313921061
:10349000121012149214CB30831692008A110A1261
:1034A000F3278A150A16031792010A127F250A16B6
:1034B0000A1272270A168A1192238A15831660113E
:1034C0008312E201E3018C1283168C16E0128B1634
:1034D0000B178B178312AC01AD0183166011E1014C
:1034E000E2015830831203179F004D30A0004E3088
:1034F000A1005B30A2005C30A3005930A4005A3018
:10350000A5000A12AF230A1658308312031792003F
:103510004D3093004E3094005B3095005C30960047
:10352000593097005A3098008A11E7218A15031301
:10353000851A9C2A08139D2A0817051AA12A8813A0
:10354000A22A8817851AA62AE101A82A0130E100DB
:10355000051AAC2AEF01AE2A0230EF0081309F003D
:10356000031792018A1100208A1583120313700831
:103570008316E3007108E4000A12BC250A16003025
:10358000F4000030F5002030F6007730F7008A11A3
:103590000A12B9228A150A1670088316E700710804
:1035A000E8007208E9007308EA00C03083120317CC
:1035B000B4008A110A1275218A150A168316630847
:1035C000831203179F0083160313640883120317E3
:1035D000A0006930A1000A122B240A1669309F004E
:1035E0000A1201250A162030B2008A110A12EC24B0
:1035F0008A150A16203083120317B2008A110A12A4
:10360000EC248A150A16203083120317B2008A119F
:103610000A12EC248A150A16C03083120317B4006C
:103620008A110A1275218A150A16831667088312F1
:10363000031792008316031368088312031793007D
:103640008316031369088312031794008316031368
:103650006A08831203179500033096000030970024
:1036600008309800003099008A117A218A15630881
:10367000831203179F008316031364088312031732
:10368000A0002E30A1000A122B240A162E309F0013
:103690008A110A1203278A150A168316031367086C
:1036A000831203179F0083160313680883120317FE
:1036B000A00083160313690883120317A100831661
:1036C00003136A0883120317A2002E30A3000330ED
:1036D000A4000A127B200A160930B2008A110A12CD
:1036E0007F228A150A162E3003179F008A110A12AC
:1036F00003278A150A160930B2008A110A127F229E
:103700008A150A168316E501E6018312051ECA2BE7
:10371000851ECA2B8316E018CA2B04308312580565
:10372000F1007108043A031DAC2B80300317B4007C
:103730008A110A1275218A150A162E3003179F0066
:103740007530A0001630A1000A12CB240A162E30C4
:103750009F000A1201250A16083003135805F100CC
:103760007108083A031DCA2B80300317B4008A1170
:103770000A1275218A150A165808031792000313B6
:103780004D080317930003134E08031794008A1182
:103790009D208A158312051A2E2C851A2E2C803016
:1037A0000317B4008A110A1275218A150A162E30E1
:1037B00003179F009730A0001630A1000A12CB24F7
:1037C0000A162E309F000A1201250A160313AC01B7
:1037D000AD018A110A12E9278A150A162E3003173D
:1037E0009F008A110A1203278A150A168A110A12E3
:1037F000E9278A150A16051E022C851E022C0130A7
:10380000F000032CF0017008031D072CFB2B83161E
:10381000E0101A30FB005E30FC006E30FD00FD0B46
:103820000F2CFC0B0F2CFB0B0F2C00008030831295
:103830000317B4008A110A1275218A150A162E3050
:1038400003179F00CA30A0001630A1000A12CB2433
:103850000A162E309F000A1201250A160313851A34
:10386000542C051E542C8316E01480308312031749
:10387000B4008A110A1275218A150A162E30031710
:103880009F00A830A0001630A1000A12CB240A160F
:10389000003003132D06031D4F2C00302C06031D92
:1038A000542C8A116F248A158316E01CD42C803086
:1038B00083120317B4008A110A1275218A150A1699
:1038C0002E3003179F00B930A0001630A1000A1255
:1038D000CB240A1603132C0803179F0003132D088B
:1038E0000317A0003930A1000A122B240A162E302B
:1038F0009F000A1201250A168A110A12E9278A1561
:103900000A162E3003179F008A110A1203278A1500
:103910000A168A110A12E9278A150A16FF30831639
:103920006305F00070088312E8002C0803179F005D
:1039300003132D080317A0007008A1000A127F23AB
:103940000A164130FC00EE30FD00FD0BA52CFC0BEF
:10395000A52C00008312AC0A0319AD0A00308316AF
:103960006305F3006408FF39F4007408F000F10106
:1039700070088312E8002C0803179F0003132D081A
:103980000317A0007008A1000A127F230A16413015
:10399000FC00EE30FD00FD0BCB2CFC0BCB2C000013
:1039A0008312AC0A0319AD0A8312051A172E851E5D
:1039B000172E8316E010803083120317B4008A118B
:1039C0000A1275218A150A162E3003179F008630B9
:1039D000A0001630A1000A12CB240A162E309F0038
:1039E0000A1201250A1664309F001630A0000A1240
:1039F0004B200A162630831203179F001630A000B2
:103A00000A124B200A160630831203132C02F3000D
:103A10000030031C013E2D02F4007308F00074080E
:103A2000F100F10CF00CF1137008E6007108E700EA
:103A3000700803179F007108A0006930A1000A12E6
:103A40002B240A1669309F008A110A1203278A154F
:103A50000A168A110A12E9278A150A16E401E501F5
:103A600000306502031D362D053064020318592D00
:103A700064080317920003136508031793000A12E2
:103A80007A270A1670080313E800700803179200DB
:103A9000693093008A11A1238A1569309F008A1129
:103AA0000A1203278A150A160313E40A0319E50A02
:103AB000302D8A110A12E9278A150A160630E40009
:103AC0000030E5002D086502031D682D2C086402F6
:103AD0000318172E06306402F3000030031C013E69
:103AE0006502F4007308F0007408F100F10CF00CAA
:103AF000F1137008E6007108E700700803179F00D3
:103B00007108A0006930A1000A122B240A1669303E
:103B10009F008A110A1203278A150A160930B2007B
:103B20008A110A127F228A150A1664080317920066
:103B300003136508031793000A127A270A16700800
:103B40000313E800E40A0319E50A64080317920066
:103B500003136508031793000A127A270A167008E0
:103B6000F300F201031368087207F00073080318EA
:103B7000013EF10070088316E3007108E40070084C
:103B8000831203179F007108A0006930A1000A1278
:103B90002B240A1669309F008A110A1203278A15FE
:103BA0000A160930B2008A110A127F228A150A16F3
:103BB00083166308F0006408F1000A12BC250A1697
:103BC0000030F4000030F5002030F6007730F700C8
:103BD0008A110A12B9228A150A1670088316E7009C
:103BE0007108E8007208E9007308EA00700883129F
:103BF00003179F007108A0007208A1007308A200BB
:103C00002E30A3000330A4000A127B200A162E30A7
:103C10009F008A110A1203278A150A168A110A12AE
:103C2000E9278A150A16E40A0319E50A622D8A11A2
:103C30000A12E9278A150A1683166308F000640839
:103C4000F100F10CF00CF113F10CF00CF113700811
:103C50008312031792000A127F250A168316601931
:103C6000322E2E2E6011E01E2A2FA0308312031751
:103C70009F008A110A1203278A150A168316031356
:103C80002008553A031D4B2E3208233A031D4B2EB4
:103C90000A12D4250A162008443A031D5D2E210875
:103CA000533A031D5D2E2208313A031D582E60162B
:103CB0002208303A031D5D2E60122008443A031D8D
:103CC000B72E21088312031792000A12B1270A1691
:103CD00070080319B72E83160313220883120317E3
:103CE00092000A12B1270A1670080319B72EA030E5
:103CF0009F008A110A121A278A150A1600307106C7
:103D0000031D842E03307006031DB72E303083163A
:103D1000031321028312C80083162208313A031DBF
:103D2000A02E83124808F1000130F0007108031939
:103D30009D2EF00D7010FF3E972E831270088804A0
:103D400083162208303A031DB72E83124808F1006B
:103D50000130F00071080319B12EF00D7010FF3E14
:103D6000AB2E83127008FF3CF00070088805031327
:103D700083162008523A031D1D2F2108443A031DC3
:103D80001D2F2208443A031D1D2FA0308312031754
:103D90009F008A110A121A278A150A160030710626
:103DA000031DD42E03307006031D1D2F0313E401E1
:103DB000E50100306502031DDF2E50306402031858
:103DC0001D2F83176408A03E84000008E600E70169
:103DD0000030E7008313660803179F00031367088A
:103DE0000317A0006930A1000A122B240A166930BB
:103DF0009F008A110A1203278A150A160930B20099
:103E00008A110A127F228A150A1607306405F1000A
:103E10006508F2000030F20500307206031D122F13
:103E200000307106031D192F8A110A12E9278A151D
:103E30000A16E40A0319E50AD92E8A110A12E9279B
:103E40008A150A168316A001E0128312CB01CC0159
:083E5000C901CA016D2A2B2FE4
:0E0FF200543469346D3465343A34203400349C
:1029FC003134363446343834373437345F34493430
:102A0C0072346434613462346F34613472346434DB
:102A1C005F3446346C346F34613474345F344C340A
:102A2C00433444345F34523453345F345034693457
:102A3C00633445344534703472346F346D345F34E0
:102A4C00323434344C3443343234353436345F34E9
:102A5C004434533431343334303437345F343134D8
:102A6C00343430343634303437342E3463340D341B
:042A7C000A340034E4
:102A800070346C346134743469346E346534203499
:102A90004D346934633472346F3463346834693468
:102AA0007034203449345234443441342034623454
:102AB0006F34613472346434203461347634653474
:102AC000633420344C344334443432347834313435
:102AD0003634203451343D34323430344D3468345B
:082AE0007A340A340D3400348D
:102AE8004D3469346B3472346F34433420343134A8
:102AF8003634463438343734373420344934523451
:102B080044344134203462346F3461347234643470
:102B18002034543465347334743473342034443476
:102B2800693476346534723473342034303437344D
:102B38002D34303436342D34323430343134343466
:062B48000D340A340034D4
:102B4E00443469346D3461346E3400344C3475342D
:102B5E006E346434693400344D3461347234643408
:102B6E00693400344D346534723463347234003455
:102B7E004A346534753464346934003456346534FB
:102B8E006E34643472340034533461346D346534CD
:102B9E006434003400340034003400340034003423
:102BAE0049346E34693474342034523454344334DA
:102BBE0020344434533431343334303437342034C5
:102BCE007034613472342034643465346634613464
:0A2BDE00753474340D340A340034E9
:102BE800523465346C3465346334743475347234F7
:102BF8006534203463346F346E34743465346E3421
:102C08007534203444345334313433343034373425
:062C18000D340A34003403
:102C1E005734723469347434653420346F346E34FE
:102C2E0020344C344334443420346C3469346E34A0
:0E2C3E0065342034233431340D340A3400342C
:102C4C004E34623420346434653420346D346F3443
:102C5C00743473342034733474346F3463346B349D
:0C2C6C006534733420343D3420340034CF
:102C78000A340D344D346934733465342034613486
:102C880020346C34273468346534753472346534D0
:0C2C9800203452345434433420340034CF
:102CA40049346E346934743420344934323443340E
:102CB40020343134303430344B3468347A340D3485
:042CC4000A3400349A
:102CC8000D340A34523465346C3469347434203425
:102CD80045344534503452344F344D342034203444
:022CE8000034B6
:102CEA004C34433444343234783431343634203436
:102CFA00B2342034553441345234543420342034DC
:022D0A00003493
:102D0C004C34653463347434753472346534203423
:102D1C0045344534703472346F346D342E34203471
:022D2C00003471
:102D2E00523441345A34203449346E346434653468
:102D3E007834203445346534703472346F346D34E5
:022D4E0000344F
:102D50005334543441345234543420347334613451
:102D60007634653445346534703472346F346D3480
:022D700000342D
:102D720053346134763465342034493464347834DD
:102D82003D3420342E342E342E342E342E3420343E
:022D920000340B
:102D94004C3443344434323478343134363420348B
:102DA400B234203455344134523454342034203431
:022DB4000034E9
:102DB600533457343234203466346F34723420340A
:102DC60049346E34693474342034523454344334C0
:022DD6000034C7
:102DD8004C34433444343234783431343634203447
:102DE800B2342034553441345234543420342034ED
:022DF8000034A5
:102DFA00313436344634383437343734203449346D
:102E0A0052344434413462346F3461347234643439
:022E1A00003482
:102E1C00523465346C3465346334743475347234C0
:102E2C00653420344434533431343334303437340F
:022E3C00003460
:102E3E0046346934733472347434203449346E3405
:102E4E0069347434203452345434433420342034AE
:022E5E0000343E
:102E60003034313432343334343435343634373426
:102E700038343934413442344334443445344634AC
:102E8000463472346534713420346B3448347A34C7
:062E90003D342034003443
:102E960049346E346934743420344C344334443405
:062EA6000D340A34003473
:102EAC00413444344334203449346E3469347434FA
:062EBC000D340A3400345D
:102EC20049346E34693474342034503457344D34B8
:062ED2000D340A34003447
:02400E007A3BFB
:020000040000FA
:10420000480065006C006C006F00200049005200FF
:1042100044004100200062006F0061007200000055
:104220005000610075006C0066006A0075006A004D
:104230006F0040006600720065006500000000002D
:104240003100360046003800370037005F00490073
:1042500072006400610062006F006100720064001F
:104260005F0046006C006F00610074005F004C004E
:10427000430044005F00520053005F00500069009B
:10428000630045004500700072006F006D005F0024
:10429000320034004C0043003200350036005F002D
:1042A0004400530031003300300037005F0031001C
:1042B000340030003600300033002E006300000070
:1042C0004D00430050003200310035003000200026
:1042D000440069007300610062006C0065006400C6
:1042E0002000420079002000520065007300650044
:1042F000740020000D000A00000000000000000013
:10430000FF00FF00FF00FF00FF00FF00FF00FF00B5
:10431000FF00FF00FF00FF00FF00FF00FF00FF00A5
:10432000FF00FF00FF00FF00FF00FF00FF00FF0095
:10433000FF00FF00FF00FF00FF00FF00FF00FF0085
:104340004D0069006B0072006F00430020003100D7
:104350003600460038003700370020004900520080
:1043600044004100200062006F00610072006400A0
:1043700020005400650073007400200050004900C4
:104380004300200045004500500052004F004D0002
:104390002000310039002D00300031002D003200A6
:1043A00030003100340020000D000A000000000041
:1043B00000000000000000000000000000000000FD
:1043C0007000610075006C0066006A0075006A008C
:1043D0006F00400066007200650065002E006600F8
:1043E00072000D000A000000FF00FF00FF00FF0048
:1043F000FF00FF00FF00FF00FF00FF00FF00FF00C5
:00000001FF
